:100000000C94F6000C9415010C9415010C94150138
:100010000C9415010C94C1030C9415010C9415015A
:100020000C9415010C9415010C9415010C941501F8
:100030000C94A5190C9415010C9415010C94150140
:100040000C94B0030C9415010C9417010C94150139
:100050000C9415010C9415010C9415010C941501C8
:100060000C9415010C9415010C9415010C941501B8
:100070000C9415010C9415010C9415010C941501A8
:100080000C9415010C9415010C9415019D0F9F0FF4
:10009000A10FA30FA50FA70FA90FAB0FAD0FAF0FA8
:1000A000B10FB30FB50FB70FB90FBB0FBD0FBF0F18
:1000B000C10FFC0FFC0FFC0FFC0FFC0FFC0FC30F5C
:1000C000C50FC70FC90FCB0FCD0FCF0FD10FD50F56
:1000D000DB0FDF0FE30FE70FEB0FEF0FF30FF50F62
:1000E000F70FF90F2A102C102E1030103210341088
:1000F000361038103A103C103E1040104210441098
:10010000461048104A104C104E1089108910891062
:100110008910891089105010521054105610581020
:100120005A105C105E10621068106C107010741021
:1001300078107C108010821084108610DF10E5107B
:10014000EB10F110F710FD10031109110F1115112B
:100150001B11211127112D11331139113F11451197
:100160004B11DD10DD10DD10DD10DD10DD10511143
:1001700057115D11631169116F1175117B11851193
:100180008F119911A311AD11B711C111CD11D31157
:10019000D911DF1120122312261229122C122F122C
:1001A0003212351238123B123E12411244124712DB
:1001B0004A124D125012531256121E121E121E12C5
:1001C0001E121E121E1259125C125F12621265126A
:1001D0006E126B1268126B126E1271127412771219
:1001E0007D127A127A127D128012831211241FBEA0
:1001F000CFEFD0E1DEBFCDBF13E0A0E0B1E0E6E994
:10020000F9E300E00BBF02C007900D92AC33B107D9
:10021000D9F716E0ACE3B3E001C01D92A237B107F5
:10022000E1F70E942F010C94C91C0C9400001F924E
:100230000F920FB60F9211240F900FBE0F901F90C8
:100240001895AC0120E030E002C02F5F3F4FFA016B
:10025000E20FF31F80818823C1F7C90108956F92CF
:100260007F928F929F92AF92BF92CF92DF92EF9246
:10027000FF920F93DF93CF9300D00F92CDB7DEB7ED
:10028000F8940E94FA080E947F0E8FEF87BB18BA7D
:100290000E94760981E897E10E94C10985E69CE009
:1002A0000E94C60981E090E00E94CB09DE01119610
:1002B000E6EFF2E083E001900D928150E1F7CE018C
:1002C00001960E94B40D80E091E00E94520E81E1FF
:1002D00091E00E944A0E82E491E00E94420E0E9448
:1002E0008A0D4C0164EF71E00E94D90960E070E072
:1002F000C4010E94FE0C3C0140E050E0BC01C4017E
:100300000E94FF092CE1A22E22E0B22ECC24DD2493
:1003100090E4E92EF12C02E021E030E041E050E0F1
:10032000B301C4010E94930C88E2A82E83E0B82E8A
:1003300021E030E041E050E0B301C4010E94CB0C69
:1003400010929A031092990310929C0310929B03AF
:100350000E94AD1A8FE784BB8AE285BB0E94CD0361
:1003600085E585BB0E94CD0315BA0E94050F0E944A
:10037000FA080E94840E7894FFCF0F931F93CF93B7
:10038000DF938C018134910510F18091A503909148
:10039000A603892BE1F41F930F938BE491E09F93C5
:1003A0008F930E94A61A1092A2031092A103109399
:1003B000A4030093A30381E090E09093A6038093AD
:1003C000A50300E410E00F900F900F900F9068E0ED
:1003D0008BE20E944309C0E0D0E00DC0E091A10390
:1003E000F091A203EC0FFD1FE551FB4F608189E204
:1003F0000E9443092196C017D10780F38091990389
:1004000090919A03019749F467E08BE20E944309B7
:1004100010929A03109299030AC063E08BE20E9443
:10042000430981E090E090939A0380939903DF91D0
:10043000CF911F910F910895CF93DF938091A503E2
:100440009091A603019709F04CC088E791E09F9333
:100450008F930E94A61A2091A1033091A20380914C
:10046000A3039091A4030F900F9028173907C8F5A4
:1004700086E991E09F938F930E94A61AC091A303EF
:10048000D091A4038091A1039091A203C81BD90B22
:100490008091A1039091A203805C9F4F9093A2034F
:1004A0008093A1030F900F90C134D1055CF08FEBC6
:1004B00091E09F938F930E94A61A80E490E00E949F
:1004C000BD010DC08BED91E09F938F930E94A61A02
:1004D000CE010E94BD011092A6031092A5030F90B9
:1004E0000F90DF91CF9108951F93CF93DF93EC018D
:1004F0001092A2031092A1031092A6031092A503DA
:100500008881182F12951F7090E09F938F93812FF1
:1005100090E09F938F9388EE91E09F938F930E943A
:10052000A61A8DB79EB706960FB6F8949EBF0FBE5B
:100530008DBF143009F445C0153050F4113019F155
:10054000113090F0123049F1133009F069C02FC01A
:10055000163009F44AC01630F0F1173009F44FC0D4
:10056000183009F05DC052C08881863041F48A811C
:10057000813009F069C0CE010E94721965C0CE01B8
:100580000E94FE0E61C088E092E09F938F930E94CC
:10059000A61ACE010E94591355C08BE192E09F9399
:1005A0008F930E94A61ACE010E94A4144BC08FE222
:1005B00092E09F938F930E94A61ACE010E94EC15A1
:1005C00041C083E492E09F938F930E94A61ACE01CC
:1005D0000E94931737C087E592E09F938F930E9404
:1005E000A61ACE010E94741A2DC08BE192E09F934F
:1005F0008F930E94A61ACE010E94A50523C08BE608
:1006000092E09F938F930E94A61A1CC083E992E008
:100610009F938F930E94A61ACE010E94591B12C06D
:100620008AEA92E09F938F930E94A61A8881809312
:10063000EB0483E08093EC041092ED0483E090E0FF
:100640000E94BD010F900F90DF91CF911F910895EF
:10065000CF93DF93EC01898190E09F938F9387EB99
:1006600092E09F938F930E94A61A80919B03909192
:100670009C030F900F900F900F90019791F58BEDC9
:1006800092E09F938F930E94A61A20E030E00F9093
:100690000F90E0919D03F0919E03E20FF31FDE01A6
:1006A000A20FB31F8C91E555FC4F80832F5F3F4F06
:1006B0002034310571F780919D0390919E03805CF9
:1006C0009F4F90939E0380939D0320919D033091B3
:1006D0009E0380919F039091A00328173907E8F1AA
:1006E00027C085EE92E09F938F930E94A61A1092E6
:1006F0009E0310929D0320E030E00F900F90E09158
:100700009D03F0919E03E20FF31FDE01A20FB31FC2
:100710008C91E555FC4F80832F5F3F4F203431058E
:1007200071F730939E0320939D038981803448F4B0
:1007300010929C0310929B038BEA93E00E94740238
:100740000CC081E090E090939C0380939B0389818F
:1007500090E09093A00380939F03DF91CF91089541
:100760001F920F920FB60F9211248F930E94CF0EFB
:100770008091450382BF8F910F900FBE0F901F9005
:1007800018951F920F920FB60F9211240E945A0EC5
:100790000F900FBE0F901F90189520E040E45CE989
:1007A000CA010197F1F72F5F2931D1F70895882306
:1007B00021F0813059F084E008958EE080936F033A
:1007C0008093700388E18AB981E008958EE0809378
:1007D00054038093550388E180939A0081E0089543
:1007E000882321F0813071F084E0089510926F0326
:1007F000109270031092900019B81AB810929500D8
:1008000081E00895109254031092550310929800BD
:100810001092990010929A0010929D0081E0089524
:10082000882321F0813039F084E0089520939000EE
:1008300069B981E00895209398006093990081E060
:100840000895623011F492E001C090E0882321F015
:10085000813061F084E0089580919500990F990F9F
:10086000990F982B9093950081E0089580919D00B9
:10087000990F990F990F982B90939D0081E00895FF
:10088000663029F0673039F0653041F402C020E06D
:1008900006C020E001C021E090E002C021E091E02C
:1008A000882321F0813069F084E0089580919500DB
:1008B000220F220F990F922B982B9093950081E095
:1008C000089580919D00220F220F990F922B982B53
:1008D00090939D0081E00895653419F06F3419F408
:1008E00005C021E001C020E090E002C021E091E0DD
:1008F000882321F0813079F084E00895809195007B
:100900002295220F207E9295907F922B982B909388
:10091000950081E0089580919D002295220F207E10
:100920009295907F922B982B90939D0081E0089553
:10093000982FFA018230A0F084E008952191992344
:1009400019F0913059F404C05D9BFECF2CB906C05C
:1009500080919B0085FFFCCF20939C0061507040EC
:100960006115710559F781E00895882321F08130E0
:1009700039F084E008955D9BFECF6CB981E0089565
:1009800080919B0085FFFCCF60939C0081E00895DF
:10099000E82FDB01823010F084E008959A0113C043
:1009A000EE2321F0E13031F084E00AC05F9BFECFFE
:1009B0008CB106C080919B0087FFFCCF80919C008A
:1009C0008D93215030401216130654F381E00895A0
:1009D000882321F0813031F084E008955F9BFECFC1
:1009E0008CB1089580919B0087FFFCCF80919C0083
:1009F000089570E00E9498048093EC041092ED0436
:100A000083E090E00E94BD0108950E94400480931D
:100A1000EC041092ED0483E090E00E94BD01089583
:100A20000E9440048093EC041092ED0483E090E077
:100A30000E94BD0108950E9421048093EC0410924D
:100A4000ED0483E090E00E94BD0108950F930E94A1
:100A500010048093EC041092ED0483E090E00E9477
:100A6000BD010F9108950E94F0038093EC04109251
:100A7000ED0483E090E00E94BD010895882321F0F9
:100A8000813051F084E011C08EE080936F03809339
:100A9000700388E18AB908C08EE080935403809384
:100AA000550388E180939A0081E08093EC041092D2
:100AB000ED0483E090E00E94BD010895CF92DF92A3
:100AC000EF92FF920F931F93DF93CF93CDB7DEB7D3
:100AD0008B01CDB6DEB62DB73EB7261B370B0FB652
:100AE000F8943EBF0FBE2DBFEDB6FEB60894E11CD4
:100AF000F11CAB01B7010E94C8048093EC0420E014
:100B000030E00AC0F701E20FF31F8081F901E351E1
:100B1000FB4F80832F5F3F4F201731079CF3F80175
:100B2000E351FB4F1082C80103960E94BD010FB62E
:100B3000F894DEBE0FBECDBECF91DF911F910F9115
:100B4000FF90EF90DF90CF9008950F93FC0180818C
:100B50008093EB048081843611F1853648F4823627
:100B6000B1F08336E0F4803651F0813681F50BC068
:100B7000873639F18836E9F0853649F515C0828126
:100B80000E943E052DC082810E94330529C0068146
:100B900025814481638182810E94260521C0638171
:100BA00082810E941B051CC0638182810E94050511
:100BB00017C0AF014C5F5F4F638182810E94F904CF
:100BC0000FC0638170E082810E945E0509C083E0EE
:100BD0008093EC041092ED0483E090E00E94BD014C
:100BE0000F91089587E28093530685E28093520621
:100BF00090E2909354061092550628E030E030932E
:100C000057062093560683E280935F0681E2809325
:100C10005E069093600610926106309363062093FF
:100C200062060895089560916B0681E20E9443096F
:100C3000089568E08BE20E94430961E188E20E9426
:100C4000430968E08FE20E94430961E18CE20E945F
:100C5000430961E08FE20E94430910929A031092C7
:100C6000990365E083E20E94430908950F931F935F
:100C70008C0160E480E20E944309F80162816058BF
:100C800084E00E944309F801828180936A061F91E3
:100C90000F9108950F931F93CF93DF93EC01288555
:100CA000398512161306DCF58E819F818217930712
:100CB0001CF568E083E20E94430900E010E00FC0E9
:100CC000EA85FB85E80FF91F608181E20E944309F4
:100CD0008E819F8101969F838E830F5F1F4F8E8130
:100CE0009F8128853985083011051CF482179307E8
:100CF0003CF38217930724F061E087E20E944309E6
:100D00008B81813031F465E089810E9443091B8227
:100D100006C061E089810E94430981E08B83DF91F5
:100D2000CF911F910F910895DF93CF9300D000D002
:100D3000CDB7DEB7FC013281238110926506109297
:100D4000640681E0809361062230F1F0233079F16E
:100D5000213009F057C080913E06809366061092BC
:100D600067068EE396E09093690680936806868115
:100D700097818034910509F045C088E090E0909318
:100D80006706809366063EC08681978190936706CA
:100D900080936606832F90E0880F991FE09150069C
:100DA000F0915106E80FF91F8081918127C033230C
:100DB000B9F0832F90E0880F991FE091A903F0917B
:100DC000AA03E80FF91F0190F081E02DF093690666
:100DD000E09368068081809366061092670612C0D1
:100DE00094E099832A8389E08B839C8384E090E05C
:100DF0009093670680936606CE01019690936906EC
:100E0000809368068EE596E00E944A060F900F9048
:100E10000F900F90CF91DF910895CF93DF9382E2EF
:100E20000E940B09C82F85FF1AC068E083E20E9468
:100E30004309C6FF10C02091640630916506809179
:100E4000660690916706281739072CF48EE596E020
:100E50000E944A0604C061E087E20E944309DF91D4
:100E6000CF9108950F931F9388E00E940B09082FDC
:100E7000182F86FF18C060E085E00E94430960E8F3
:100E800084E00E94430960E080E20E94430968E038
:100E900083E20E94430961E087E20E94430962E025
:100EA00085E00E94430914FF04C060EC89E00E94C1
:100EB000430907FF04C060ED89E00E9443091F91C8
:100EC0000F9108958AE00E940B0980FF03C00E94E1
:100ED0000D07089581FF0DC08AE20E940B098091E1
:100EE0002B06813061F4E0912E06F0912F060995D2
:100EF000089582E30E940B098AE30E940B0908957A
:100F00008EE00E940B0968E08FE20E94430961E0D5
:100F10008FE20E9443092091660630916706809116
:100F2000620690916306821793075CF468E083E29F
:100F30000E94430961E087E20E94430981E08093B7
:100F400061060895EF92FF920F931F93DF93CF9363
:100F5000CDB7DEB728970FB6F894DEBF0FBECDBF72
:100F600086E20E940B0986FF7FC08E010F5F1F4F34
:100F700049E0E42EF12CEC0EFD1E809152060E94F9
:100F80000B09F80181938F01EE15FF05B1F78E0172
:100F90000F5F1F4F68E087E20E94430968E083E229
:100FA0000E94430980E20E940B098F77682F80E23C
:100FB0000E944309898190E080769070803291058B
:100FC00009F440C080349105D1F1892BF1F5F80185
:100FD00081818630D9F0873048F48130F1F1813059
:100FE000C8F08330D1F1853081F521C0893019F105
:100FF0008A3018F4883049F505C08A3071F18B3099
:1010000021F520C060916B0681E225C0C8010E94D5
:10101000940623C068E083E20E94430961E081E214
:101020000E94430960E081E20E9443090BC0C801AD
:101030000E94360612C0C8010E9419060EC0C801DF
:101040000E94F80865E083E206C080E20E940B0976
:101050008058682F80E20E944309F801808188232C
:10106000D1F465E083E215C02091660630916706F1
:1010700080916206909163068217930764F4109240
:1010800067061092660668E083E20E94430961E009
:1010900087E20E94430928960FB6F894DEBF0FBE80
:1010A000CDBFCF91DF911F910F91FF90EF900895E9
:1010B000EF92FF920F931F93DF93CF93CDB7DEB7DD
:1010C000C054D0400FB6F894DEBF0FBECDBF8CE049
:1010D0000E940B0980FF03C00E94A2077BC081FF12
:1010E0002AC08EE20E940B098DE20E940B098983BF
:1010F0008E010F5F1F4F70E4E72EF12CEC0EFD1EEA
:101100000F5F1F4F0E943009F80180830E151F05E5
:10111000B9F780913C03813039F4E0913F03F091BD
:101120004003CE010196099568E08FE20E944309D1
:1011300061E08FE22BC082FF2CC086E30E940B0986
:1011400085E30E940B0989838E010F5F1F4F60E4C6
:10115000E62EF12CEC0EFD1E0F5F1F4F0E94300992
:10116000F80180830E151F05B9F780913D0381308A
:1011700039F4E0914103F0914203CE0101960995C3
:1011800068E087E30E94430961E087E30E94430926
:1011900021C083FF1FC08EE30E940B098E010F5FE9
:1011A0001F4F51E4E52EF12CEC0EFD1E8DE30E9445
:1011B0000B09F80181938F01EE15FF05B9F78091B6
:1011C0003E03813039F4E0913F03F0914003CE01BA
:1011D00001960995C05CDF4F0FB6F894DEBF0FBED5
:1011E000CDBFCF91DF911F910F91FF90EF900895A8
:1011F0000895089581E08ABF80E189BFE4E6F0E0C8
:10120000808187608083E5E6F0E080818360808371
:10121000A79AAF9A08959FEF9ABB8BBB85B380586E
:1012200085BBE5E6F0E0808195E08927808385B382
:10123000805885BB80818927808300001ABA85B3D6
:10124000805885BB808122E08227808300000000D7
:1012500089B395B3905895BB908192279083089558
:1012600085B3805885BBE5E6F0E0808122E08227E7
:1012700080830000000089B395B3905895BB90819E
:101280009227908308958BBB8FEF8ABB85B38058DC
:1012900085BBE5E6F0E0808195E08927808385B312
:1012A000805885BB8081892780836BBB85B380583C
:1012B00085BB808191E08927808385B3805885BB79
:1012C00080818927808308958BBB85B3805885BB37
:1012D000E5E6F0E0808191E08927808385B380583E
:1012E00085BB8081892780830895089582E180935A
:1012F0003E0681E080933F0680E191E090934106B5
:1013000080934006109242061092430610924406C3
:1013100088E0809345061092470610924606109288
:1013200049061092480610924B0610924A061092F7
:101330004C0610924D0610924E0610924F061092D7
:101340003C0310923D0310923E0310922B06109224
:101350002C0610922D06109235061092340610922B
:10136000A8031092A703089590934706809346061A
:10137000709349066093480650934B0640934A0683
:1013800008959093470680934606089590934906E2
:1013900080934806089590934B0680934A060895DB
:1013A00080934206089580934306089580934406EF
:1013B00008950F931F93CF93DF938C01CB01C091BE
:1013C0003406D091350662E070E00E94A21C10C085
:1013D000988129818A81823041F4E92FF22F858119
:1013E00090E08017910709F460870F80D885C02DA1
:1013F000209771F7DF91CF911F910F910895CF93AF
:10140000DF939C01E0913406F091350614C0A08171
:10141000B1818281843061F4848190E082179307E6
:1014200039F4868190E08617970711F4ED014B831C
:101430000780F085E02D309751F7DF91CF91089527
:101440008F929F92BF92CF92DF92EF92FF920F9373
:101450001F93CF93DF934C01F62ED42EC22EB02EC5
:10146000E0913406F0913506309799F489E090E0E8
:101470000E94A31BFC019093350680933406918251
:101480008082F38210861782D282C4820583E6822C
:1014900018C0CF010780F085E02D3097D1F78C017F
:1014A00089E090E00E94A31BFC01E80198878F83EC
:1014B00091828082F382D282C482B582E6821086D3
:1014C0001782DF91CF911F910F91FF90EF90DF90E6
:1014D000CF90BF909F908F900895EF92FF921F93AF
:1014E000CF93DF937C01C091A703D091A8032097ED
:1014F00011F011E012C085E090E00E94A31BFC01F6
:101500009093A8038093A703F182E0821282148251
:10151000138210E012C01F5FEC018B819C81009749
:10152000D1F785E090E00E94A31BFC019C838B8394
:10153000F182E082128314821382812FDF91CF9196
:101540001F91FF90EF900895EF92FF920F931F93DA
:10155000CF93DF93E091A703F091A80380E090E0A0
:101560000380F481E02D01963097D1F7880F991F01
:101570000E94A31B8093A9039093AA03C091A70381
:10158000D091A80301C0EC01E880F9808A8190E045
:10159000880F991F0091A9031091AA03080F191F22
:1015A000F701808190E00E94A31BF8018083918362
:1015B00020E030E016C08A8190E0880F991FE0910A
:1015C000A903F091AA03E80FF91F0190F081E02D23
:1015D000E20FF31FD701A20FB31F8C9180832F5FFF
:1015E0003F4FF701808190E02817390724F38B8162
:1015F0009C81009741F6DF91CF911F910F91FF9051
:10160000EF9008956F927F928F929F92AF92BF92C8
:10161000CF92DF92EF92FF920F931F93CF93DF93BE
:10162000E0913406F0913506CC24DD2409C0828196
:10163000823019F40894C11CD11C0780F085E02D7C
:101640003097A9F7C601880F991F0E94A31B8093AA
:101650005006909351060894C108D1085601AA0C6F
:10166000BB1C0894C11CD11CB1E06B2E712C8824CA
:10167000992451C0E0913406F0913506A9E0EA2E94
:10168000F12C15C0A081B181848190E08615970569
:1016900019F48381E80EF11CED018D81861521F48A
:1016A0008281823009F44D010780F085E02D30976A
:1016B00049F700915006109151060A0D1B1DC701F4
:1016C0000E94A31BF8018083918320E030E0E09129
:1016D0005006F0915106EA0DFB1D0190F081E02DBE
:1016E000E20FF31FD401A20FB31F8C9180832F5FF1
:1016F0003F4F2930310559F7E0915006F0915106DE
:10170000EA0DFB1D0190F081E02D8E2D875F828315
:101710000894611C711CC614D7040CF0ABCFE1E037
:10172000EE2EF12C79E0A72EB12C662477248824A4
:10173000992499C0A0913406B091350612C0ED915C
:10174000FC9111978181823049F4858190E08E155A
:101750009F0521F48481682E772405C0ED01AF81B7
:10176000B885109761F701E010E072C0409134062F
:101770005091350667C0DA01ED91FC91818184308A
:1017800009F05DC0EA018E8190E08017910709F0B1
:1017900056C08C8190E08E159F0509F050C0DF0186
:1017A0009501BF01675F7F4FE0915006F0915106B0
:1017B000E80DF91D0190F081E02DE20FF31F8D91EE
:1017C00080832F5F3F4FA617B70771F7E9E0F0E07E
:1017D000AE0EBF1EA0913406B09135062EC0ED01AD
:1017E0008A81853039F58C8190E08E159F0511F541
:1017F0008D8190E080179107E9F4CD91DC911197EC
:101800009501BE01695F7F4FE0915006F09151064E
:10181000E80DF91D0190F081E02DE20FF31F899191
:1018200080832F5F3F4FC617D70771F7E7E0F0E0DF
:10183000AE0EBF1EED01AF81B885109781F6FA019B
:10184000478150854115510509F095CF0F5F1F4F16
:10185000601671060CF08ACF0894E11CF11C82E03E
:1018600090E0880E991ECE14DF040CF063CFDF9158
:10187000CF911F910F91FF90EF90DF90CF90BF908D
:10188000AF909F908F907F906F9008958F929F92CE
:10189000AF92BF92CF92EF92FF920F931F93CF938D
:1018A000DF935C014B01122FE0913406F091350675
:1018B00016C0A081B181848190E0A816B90661F4B8
:1018C000868190E08815990539F48281843021F46D
:1018D000ED018C818F5F8C830780F085E02D309740
:1018E00041F787E090E00E94A31BFC0187E0808322
:1018F00085E0818312830383F582E482C682EE242D
:10190000082D2A2D45E067E0CF010E94200ADF91D3
:10191000CF911F910F91FF90EF90CF90BF90AF901C
:101920009F908F900895AF92BF92CF92DF92EF92E7
:10193000FF920F93FC01A114B10401F14230510553
:1019400071F04330510599F041305105B9F481E00F
:1019500080932B06B0922F06A0922E060FC081E036
:1019600080932C06B0923106A092300607C081E029
:1019700080932D06B0923306A092320620583F4F36
:10198000CF010E94460C0F91FF90EF90DF90CF9017
:10199000BF90AF900895AF92BF92CF92DF92EF9237
:1019A000FF920F93FC014230510571F04330510515
:1019B00099F041305105B9F481E080933C03B09235
:1019C0004003A0923F030FC081E080933D03B0929B
:1019D0004203A092410307C081E080933E03B0928E
:1019E0004403A0924303CF010E94460C0F91FF9045
:1019F000EF90DF90CF90BF90AF900895EF920F934C
:101A00001F93CF93DF93182F062FA0913406B09128
:101A10003506C0E0D0E014C02D913C911197F9013A
:101A20008581811751F4FD018281823031F4F90101
:101A300084818F5F8483C82FD0E0FD01A781B085AA
:101A4000109751F789E090E00E94A31BFC0189E008
:101A5000808384E08183028313821482158216823C
:101A600017821086EC2E00E0212F44E069E0CF01C0
:101A70000E94200ACE01DF91CF911F910F91EF902C
:101A80000895DF92EF92FF920F931F93CF93DF930E
:101A9000182FE62EF42ED22EA0913406B0913506E2
:101AA000C0E0D0E014C02D913C911197F9018581DF
:101AB000811751F4FD018281823031F4F901848172
:101AC0008F5F8483C82FD0E0FD01A781B085109778
:101AD00051F789E090E00E94A31BFC0189E080831C
:101AE00084E08183E28213821482F582D6820783A6
:101AF0001086EC2E00E0212F44E069E0CF010E9427
:101B0000200ACE01DF91CF911F910F91FF90EF90AE
:101B1000DF900895EF920F931F9310914F061F5F70
:101B200010934F0689E090E00E94A31BFC0189E01E
:101B3000808389E090E09383828382E081831482B2
:101B40001583168280EA87838AE18087EE2400E08D
:101B500020E042E069E0CF010E94200A812F90E05E
:101B60001F910F91EF9008950F931F93CF93DF93E1
:101B70008C01FC0101900020E9F7E81BF90BCF0173
:101B8000880F991F0E94A31BEC01F801019000200F
:101B9000E9F7E01BF10BEE0FFF1FE88323E0298339
:101BA000AC0120E030E009C0F801E20FF31F8081B2
:101BB000FA01808311822F5F3F4FF80101900020CE
:101BC000E9F73197E01BF10B4E5F5F4F2E173F0790
:101BD00058F3CE010E946D0A90E0DF91CF911F91E2
:101BE0000F910895EF92FF920F931F93CF93DF937E
:101BF0008C017B01CA010E94B40D282FE0913406AC
:101C0000F091350614C0A081B1818281843061F4E5
:101C1000848190E08017910739F4868190E08E15D9
:101C20009F0511F4ED0128870780F085E02D30979E
:101C300051F7DF91CF911F910F91FF90EF90089591
:101C4000CF93DF93EC01CB010E94B40D382FA0910C
:101C50003406B091350611C09C91FD01218182812D
:101C6000823041F4E92FF22F858190E08C179D0797
:101C700009F43683FD01A781B085109769F7DF91DC
:101C8000CF9108950E94B40D1816190614F480938C
:101C90004E0608950E94B40D1816190614F4809388
:101CA0004D0608950E94B40D1816190614F4809379
:101CB0004C0608951F9386E00E940B0986FF03C01F
:101CC0000E9458080EC082FF03C00E94620709C02C
:101CD00081FF03C00E94320704C084FF02C00E943B
:101CE000800787E00E940B09182F60E087E00E94C0
:101CF0004309612F87E00E9443091F91089562E024
:101D000081E00E94430908950E94020B0E94A40AE8
:101D10000E94F20561E080E00E94430980E00E9499
:101D20000B0980FDFBCF62E081E00E94430960E87F
:101D300084E00E94430960E480E20E94430968E075
:101D400083E20E94430969E087E20E9443096FE051
:101D50008DE00E9443096FE08BE00E94430968ED2B
:101D600089E00E94430963E38FE00E94430966ED26
:101D700087E00E94430962E085E00E9443096CEC21
:101D800080E00E94430908958EEC8093450381E032
:101D900087BF8091450382BF83E083BF0895089584
:101DA000089583E08093EB0481E08093EC048BE062
:101DB0008093ED049FE69093EE0483E68093EF0416
:101DC00084E78093F0049093F10480E78093F20419
:101DD00085E78093F30483E78093F4048FE5809391
:101DE000F50480E38093F60481E38093F704109276
:101DF000F8048EE090E00E94BD010895FC0180810E
:101E0000833011F40E94D10E08951F9311E0812FA9
:101E10000E94FE0F60E0812F0E94C4101F5F1431EA
:101E2000B1F718E1812F0E94FE0F60E0812F0E9420
:101E3000C4101F5F1B32B1F71F910895FC0110827F
:101E400075836483738362834183478346830895E4
:101E5000FC0190818181981710F080E00895A481A1
:101E6000B5816D938781815019F48181A81BB109D7
:101E70008783B583A4839FB7F89480818F5F808325
:101E80009FBF81E00895FC0180818823E9F3A2814E
:101E9000B3812D918681815019F48181A81BB109EC
:101EA000B383A28386839FB7F89480818150808317
:101EB0009FBF822F0895FC018081882319F42FEFA2
:101EC0003FEF13C0A281B3812D918681815019F417
:101ED0008181A81BB109B383A28386839FB7F8943D
:101EE0008081815080839FBF30E0C901089581E0E7
:101EF000089581E0089581E0089581E00895982F84
:101F00008150833120F08751833108F075C0E92F6B
:101F1000F0E0EB5BFC4F82E08183892F90E0FC01D5
:101F20003197EC32F10508F067C0EA5BFF4FEE0F26
:101F3000FF1F0590F491E02D0994159A5BC0169A45
:101F400059C0179A57C0B89A55C0B99A53C0BA9A8F
:101F500051C0BB9A4FC0BC9A4DC0BD9A4BC0BE9AEF
:101F600049C0BF9A47C0889A45C0899A43C08A9A97
:101F700041C08B9A3FC08C9A3DC08D9A3BC08E9ACF
:101F800039C08F9A37C0A09A35C0A19A33C0A29A9F
:101F900031C0A39A2FC0A49A2DC0A59A2BC0A69A8F
:101FA00029C080916100806803C0809161008064D5
:101FB000809361001FC0809161008062F9CF8091A1
:101FC00061008061F5CF809161008860F1CF8091E0
:101FD00061008460EDCF809161008260E9CF8091E3
:101FE00061008160E5CF109A05C0119A03C0129A72
:101FF00001C0139A81E0089584E00895982F8150DC
:10200000833128F08751833110F084E00895892FBF
:102010000E947F0F81E00895982F8150833120F036
:102020008751833108F075C0E92FF0E0EB5BFC4F7E
:1020300081E08183892F90E0FC013197EC32F1053A
:1020400008F067C0EE58FF4FEE0FFF1F0590F491A8
:10205000E02D099415985BC0169859C0179857C081
:10206000B89855C0B99853C0BA9851C0BB984FC0E2
:10207000BC984DC0BD984BC0BE9849C0BF9847C0E2
:10208000889845C0899843C08A9841C08B983FC0C2
:102090008C983DC08D983BC08E9839C08F9837C0C2
:1020A000A09835C0A19833C0A29831C0A3982FC082
:1020B000A4982DC0A5982BC0A69829C08091610036
:1020C0008F7703C0809161008F7B809361001FC078
:1020D000809161008F7DF9CF809161008F7EF5CF77
:1020E00080916100877FF1CF809161008B7FEDCF80
:1020F000809161008D7FE9CF809161008E7FE5CF77
:10210000109805C0119803C0129801C0139881E07F
:10211000089584E00895FB011082833089F08430B3
:1021200028F4813049F0823029F408C0843051F01D
:10213000853051F085E0089586B307C083B305C0AC
:1021400080B303C081B101C080B1808381E0089574
:10215000833089F0843028F4813049F0823029F4CA
:1021600008C0843051F0853059F084E0089568BB90
:1021700005C065BB03C062BB01C063B981E00895BF
:102180006093620081E00895982FE82FF0E0EB5B08
:10219000FC4F8181823011F086E00895892F90E014
:1021A000FC013197EC32F10540F4E256FF4FEE0F9F
:1021B000FF1F0590F491E02D099484E008956623B3
:1021C00011F01D9AFFC01D98FDC0662311F01E9AE4
:1021D000F9C01E98F7C0662311F01F9AF3C01F982C
:1021E000F1C0662311F0C09AEDC0C098EBC0662321
:1021F00011F0C19AE7C0C198E5C0662311F0C29AF8
:10220000E1C0C298DFC0662311F0C39ADBC0C39857
:10221000D9C0662311F0C49AD5C0C498D3C0662330
:1022200011F0C59ACFC0C598CDC0662311F0C69AEB
:10223000C9C0C698C7C0662311F0C79AC3C0C79863
:10224000C1C0662311F0909ABDC09098BBC06623B0
:1022500011F0919AB7C09198B5C0662311F0929A87
:10226000B1C09298AFC0662311F0939AABC0939817
:10227000A9C0662311F0949AA5C09498A3C06623C0
:1022800011F0959A9FC095989DC0662311F0969A7B
:1022900099C0969897C0662311F0979A93C0979823
:1022A00091C0662311F0A89A8DC0A8988BC06623B0
:1022B00011F0A99A87C0A99885C0662311F0AA9A3F
:1022C00081C0AA987FC0662311F0AB9A7BC0AB98FF
:1022D00079C0662311F0AC9A75C0AC9873C06623C0
:1022E00011F0AD9A6FC0AD986DC0662311F0AE9A33
:1022F00069C0AE9867C0662321F080916200806853
:1023000049C0809162008F7745C0662321F080919B
:10231000620080643FC0809162008F7B3BC0662377
:1023200021F080916200806235C0809162008F7DD3
:1023300031C0662321F08091620080612BC08091C2
:1023400062008F7E27C0662321F080916200886042
:1023500021C080916200877F1DC0662321F080919B
:102360006200846017C0809162008B7F13C0662377
:1023700021F08091620082600DC0809162008D7FAB
:1023800009C0662321F080916200816003C08091C2
:1023900062008E7F8093620015C0662311F0189A48
:1023A00011C018980FC0662311F0199A0BC0199824
:1023B00009C0662311F01A9A05C01A9803C0662353
:1023C00019F01B9A81E008951B9881E008951F93EE
:1023D000182F8150833128F08751833110F084E029
:1023E0000EC0E12FF0E0EB5BFC4F83E08183812F97
:1023F0000E947F0F61E0812F0E94C41081E01F9135
:102400000895CF93DF93982FEB011882E82FF0E027
:10241000EB5BFC4F8181813011F086E07AC0892F1F
:1024200090E0FC013197EC32F10540F4E653FF4FA8
:10243000EE0FFF1F0590F491E02D099484E069C030
:102440000D9B66C062C00E9B63C05FC00F9B60C0E7
:102450005CC0B09B5DC059C0B19B5AC056C0B29B16
:1024600057C053C0B39B54C050C0B49B51C04DC063
:10247000B59B4EC04AC0B69B4BC047C0B79B48C037
:1024800044C0809B45C041C0819B42C03EC0829BEE
:102490003FC03BC0839B3CC038C0849B39C035C023
:1024A000859B36C032C0869B33C02FC0879B30C00F
:1024B0002CC0989B2DC029C0999B2AC026C09A9BEE
:1024C00027C023C09B9B24C020C09C9B21C01DC053
:1024D000079B1EC01AC0069B1BC017C0059B18C0D7
:1024E00014C0049B15C011C0039B12C00EC0029BF8
:1024F0000FC00BC0089B0CC008C0099B09C005C0D9
:102500000A9B06C002C00B9B03C081E0888301C008
:1025100081E0DF91CF910895DF93CF930F92CDB7F4
:10252000DEB79BE19093EB04BE016F5F7F4F0E948B
:1025300001128093EC0489818093ED041092EE04E3
:1025400084E090E00E94BD010F90CF91DF9108954B
:102550009AE19093EB040E94C4108093EC041092D3
:10256000ED0483E090E00E94BD01089598E190930E
:10257000EB040E94A8108093EC041092ED0483E019
:1025800090E00E94BD010895982F89E18093EB04AB
:10259000933091F0943028F4913051F0923029F436
:1025A00009C0943059F0953059F085E090E00AC0A8
:1025B00096B307C093B305C090B303C091B101C0F7
:1025C00090B181E08093EC049093ED041092EE04BE
:1025D00084E090E00E94BD01089597E19093EB04A0
:1025E0000E94E7118093EC041092ED0483E090E0E8
:1025F0000E94BD01089595E19093EB040E940C1098
:102600008093EC041092ED0483E090E00E94BD0101
:10261000089596E19093EB040E947F0F8093EC0461
:102620001092ED0483E090E00E94BD01089584E1E2
:102630008093EB0481E08093EC041092ED0483E03E
:1026400090E00E94BD01089582E18093EB0481E057
:102650008093EC041092ED0483E090E00E94BD01B1
:10266000089583E18093EB0481E08093EC04109261
:10267000ED0483E090E00E94BD01089580E1809325
:10268000EB0481E08093EC041092ED0483E090E091
:102690000E94BD01089591E19093EB040E94FE0F0A
:1026A0008093EC041092ED0483E090E00E94BD0161
:1026B0000895FC0180818531C9F1863180F4823131
:1026C00031F1833130F48031D1F0813109F04CC0E7
:1026D0001AC0833109F1843109F046C022C0883123
:1026E00089F1893128F4863129F18731E9F526C04D
:1026F0008A3189F18A3158F18B31B1F531C082814B
:102700000E943E13089582810E944B1308956381B5
:1027100082810E9424130895638182810E94311373
:102720000895638182810E941713089582810E9417
:10273000FB12089582810E940913089582810E94EC
:10274000ED120895638182810E94B61208958281FC
:102750000E94C4120895638182810E94A812089584
:1027600082810E948C1208958093EB0483E0809311
:10277000EC041092ED0483E090E00E94BD01089506
:10278000E82F8152883018F024E030E007C0F0E0F4
:10279000EB5BFC4F84E0818321E030E0C9010895C8
:1027A000E82FF0E0EB5BFC4F8181843019F024E0EE
:1027B00030E003C0118221E030E0C901089517B86C
:1027C000823039F0833039F0813041F022E030E05E
:1027D00007C03E9A03C087B1806C87B921E030E022
:1027E000C901089593E896B997B1907F982B97B94E
:1027F000369A3699FECF84B195B140E050E020E0A2
:1028000030E0369A3699FECF84B195B1280F391F42
:102810004F5F5F4F44305105A1F7379836952795A4
:1028200036952795C9010895CF93DF93EB0119825F
:102830001882282F30E0F901EB5BFC4F8181843056
:1028400019F026E030E00AC088E290E0821B930B8A
:102850000E94F2139983888321E030E0C901DF915F
:10286000CF910895982F83E28093EB0417B89230AC
:1028700039F0933039F0913041F082E090E007C0B8
:102880003E9A03C087B1806C87B981E090E0809365
:10289000EC041092ED0483E090E00E94BD010895E5
:1028A000DF93CF9300D0CDB7DEB792E29093EB04E5
:1028B000BE016F5F7F4F0E9414148093EC049981D6
:1028C0008A818093ED049093EE041092EF0485E0EA
:1028D00090E00E94BD010F900F90CF91DF9108957D
:1028E00091E29093EB04E82FF0E0EB5BFC4F8181E9
:1028F000843019F084E090E003C0118281E090E020
:102900008093EC041092ED0483E090E00E94BD01FE
:102910000895E82F80E28093EB048E2F8152883057
:1029200018F084E090E007C0F0E0EB5BFC4F84E03F
:10293000818381E090E08093EC041092ED0483E0C9
:1029400090E00E94BD010895FC018081813271F008
:10295000823218F48032B1F405C0823259F08332E9
:1029600089F40CC082810E948914089582810E949A
:102970007014089582810E945014089582810E94EB
:10298000321408958093EB0483E08093EC0410925A
:10299000ED0483E090E00E94BD01089584E08093FF
:1029A0007400109271008BE0809352038CE080934E
:1029B000530381E090E00895E4E7F0E080818B7FAD
:1029C0008083109252031092530381E090E00895A7
:1029D00080937000E1E7F0E080818C7F808381E06C
:1029E00090E0089580917100887F0895982F84EA7F
:1029F000809374008091740087FFFCCF80917100F8
:102A0000887F883011F0803181F49093730084E8DE
:102A1000809374008091740087FFFCCF80917100D7
:102A2000887F883129F0803419F022E030E002C03C
:102A300021E030E0C901089584E980937400809119
:102A4000740084FDFCCF81E090E00895AC0120E0AB
:102A500030E094E812C0FA01E20FF31F8081809306
:102A600073009093740080917100887F883219F010
:102A700022E030E007C02F5F3F4F261737075CF397
:102A800021E030E0C901089584EC809374008091C6
:102A9000740087FFFCCF80917300089585E38093D5
:102AA000EB0481E08093EC0420E030E094EC0EC075
:102AB000909374008091740087FFFCCF8091730025
:102AC000F901E351FB4F80832F5F3F4F26173707F4
:102AD0007CF3FB01E351FB4F1082CB0103960E9474
:102AE000BD010895AC0120E030E094E812C0FB0184
:102AF000E20FF31F808180937300909374008091A4
:102B00007100887F883219F082E090E007C02F5F63
:102B10003F4F241735075CF381E090E08093EC048D
:102B20001092ED0483E090E00E94BD01089584E9D5
:102B3000809374008091740084FDFCCF81E08093C9
:102B4000EC041092ED0483E090E00E94BD01089532
:102B50000E94F6148093EC041092ED0483E090E060
:102B60000E94BD01089580937000E1E7F0E080814C
:102B70008C7F808381E08093EC041092ED0483E0ED
:102B800090E00E94BD010895E4E7F0E080818B7F32
:102B90008083109252031092530381E08093EC04DF
:102BA0001092ED0483E090E00E94BD01089584E05E
:102BB00080937400109271008BE0809352038CE03C
:102BC0008093530381E08093EC041092ED0483E042
:102BD00090E00E94BD010895FC0180818093EB0488
:102BE00080818433D1F0853338F4813379F08233B6
:102BF00081F0803341F507C08633F1F08633A8F0C9
:102C0000873309F51DC00E94D71508950E94C41589
:102C1000089582810E94B3150895BF016D5F7F4FB3
:102C2000828190E00E9472150895638170E0828134
:102C300090E00E944E15089582810E94A815089583
:102C40000E949715089583E08093EC041092ED04A0
:102C500083E090E00E94BD010895782F613041F03B
:102C6000613040F0623041F0633009F059C007C074
:102C700060E006C060E001C061E050E002C061E0D9
:102C800051E04330B9F0443028F4413059F042303B
:102C900078F40AC0453099F0453070F0463009F0BC
:102CA0003FC010C021E00CC021E041E030E00DC089
:102CB00021E009C020E0F9CF20E041E005C020E09C
:102CC00040E0F4CF20E040E031E0BB9887B386607D
:102CD00087BB88B3817F88BB80E090E0772311F0C9
:102CE00081E090E075E0880F991F7A95E1F78065A3
:102CF000660F660F660F682B550F550F562B542B1A
:102D0000220F252B2DB93EB988E080934B038AE032
:102D100080934C0389E080934D0321E030E002C0B2
:102D200022E030E0C90108951DB81EB810924B038F
:102D300010924C0310924D0381E090E00895AC0195
:102D400020E007C0E60FF71F80818FB9779BFECF89
:102D50002F5FE22FF0E0E417F507A4F381E090E0A5
:102D60000895DC0120E030E040E050E013C01FB8DF
:102D700008C083E0493E580714F088E008954F5F8B
:102D80005F4F779BF6CF8FB1FB01E20FF31F80837C
:102D90002F5F3F4F2A173B0754F381E00895CF93ED
:102DA000DF93EC0120E030E0A0E0B0E017C0FE01CE
:102DB000E20FF31F80818FB908C0119683E0A93E0E
:102DC000B8071CF028E030E00EC0779BF6CF8FB13B
:102DD000FB01E20FF31F80832F5F3F4F241735075E
:102DE00034F321E030E0C901DF91CF910895DC0197
:102DF00083E48093EB0440E050E020E030E018C032
:102E0000FD01E20FF31F80818FB909C04F5F5F4F53
:102E100083E0493E58071CF028E030E00EC0779B65
:102E2000F5CF8FB1F901E551FB4F82832F5F3F4F03
:102E3000261737072CF321E030E02093EC04FB0148
:102E4000E351FB4F1082CB0103960E94BD01089510
:102E5000BC0184E48093EB0440E050E020E030E0EB
:102E600013C01FB808C083E0493E580714F088E03B
:102E70000FC04F5F5F4F779BF6CF8FB1F901E551E0
:102E8000FB4F82832F5F3F4F2617370754F381E0B4
:102E90008093EC04FB01E351FB4F1082CB010396BE
:102EA0000E94BD01089593E49093EB04282F30E035
:102EB00090E007C0E60FF71F80818FB9779BFECFA8
:102EC0009F5FE92FF0E0E217F307A4F381E080931E
:102ED000EC041092ED0483E090E00E94BD0108959F
:102EE00081E48093EB041DB81EB810924B0310923E
:102EF0004C0310924D0381E08093EC041092ED049A
:102F000083E090E00E94BD01089590E49093EB046B
:102F10000E942D168093EC041092ED0483E090E063
:102F20000E94BD010895CF93DF93EC018881833423
:102F3000A9F0843428F4803441F0813409F50BC0C1
:102F4000843499F08534E1F414C04C816B818A811A
:102F50000E94851720C00E9470171DC0BE016D5FC2
:102F60007F4F8A810E94531716C08A8190E00E9489
:102F700028176A8170E0CE0103960E94F7160BC0F5
:102F80008093EB0483E08093EC041092ED0483E0E3
:102F900090E00E94BD01DF91CF910895B89AB99A4F
:102FA000BA9ABB98BC9ABD9AC498C59881E08093A0
:102FB000560382E08093570380935803809359030C
:102FC00081E090E0089510925603109257031092FA
:102FD00058031092590381E090E00895C098C19879
:102FE000C29880E29EE40197F1F7C09A8AE0982F98
:102FF0009A95F1F7C29AC19A8A95F1F70895282F08
:10300000C19887FD02C0C29801C0C29A8AE0982F79
:103010009A95F1F7C19A8A95F1F7C19826FF02C0F7
:10302000C29A01C0C2988AE0982F9A95F1F7C19A86
:103030008A95F1F70895880F20E03AE0C19887FF5C
:1030400002C0C29A01C0C298932F9A95F1F7C19A13
:10305000932F9A95F1F72F5F273011F0880FEECF5D
:10306000089520E03AE0C19887FF02C0C29A01C0EB
:10307000C298932F9A95F1F7C19A932F9A95F1F7E9
:103080002F5F283011F0880FEECF0895C198C298B5
:103090008AE0982F9A95F1F7C19A982F9A95F1F7AF
:1030A000C198C098982F9A95F1F7C19A982F9A9540
:1030B000F1F7C1988A95F1F7C09A80E00895C19818
:1030C000C098C298C39A08950E94EE1780E30E94A8
:1030D000FF1780E60E941B1808950E94EE1780E0FB
:1030E0000E94FF1780E00E941B18C198C098C298E8
:1030F000C39A08950F931F93182F062F0E94EE175F
:1031000080E40E94FF17812F0E941B18802F0E94CD
:10311000311881E01F910F9108951F93182F0E947D
:10312000EE1780EC0E94FF17812F0E941B180E944F
:1031300046181F910895C1988AE08A95F1F7C298C0
:1031400020E080E04AE0880FC19A942F9A95F1F729
:10315000C198B3998F5F3AE0942F9A95F1F72F5F5A
:10316000283089F7C098C19A932F9A95F1F7C09AA1
:10317000C198932F9A95F1F708951F93182F0E94E5
:10318000EE1780E80E94FF17812F0E941B180E94F3
:103190009B181F910895DF92EF92FF920F931F9358
:1031A000CF93DF93D82E7B018A01C0E0D0E009C025
:1031B0008D2D8C0F0E94BD18F801EC0FFD1F808330
:1031C0002196CE15DF05A0F381E090E0DF91CF914D
:1031D0001F910F91FF90EF90DF9008950F931F9331
:1031E000082F162F0E946418612F802F0E947A18D2
:1031F00081E01F910F910895DF92EF92FF920F935C
:103200001F93CF93DF93D82E7B018A01C0E0D0E0DB
:1032100009C0F801EC0FFD1F60818D2D8C0F0E94FD
:10322000EE182196CE15DF05A0F381E090E0DF9146
:10323000CF911F910F91FF90EF90DF90089594E050
:103240009093EB040E94FC188093EC041092ED0420
:1032500083E090E00E94BD010895EF92FF920F93EA
:103260001F938B019BEEE92E94E0F92E93E090934F
:10327000EB04A7014E5F5F4F0E94CB188093EC04D4
:103280000E5F1F4FE00EF11EF7011082C80101967C
:103290000E94BD011F910F91FF90EF90089582E071
:1032A0008093EB0410925603109257031092580328
:1032B0001092590381E08093EC041092ED0483E0B6
:1032C00090E00E94BD01089581E08093EB040E948C
:1032D000CE178093EC041092ED0483E090E00E94FE
:1032E000BD010895FC018381823069F0833018F4B8
:1032F0008130F1F405C0833049F08430C9F40FC047
:103300000E94641908950E944F190895AF014A5F01
:103310005F4F658170E084810E942D190895AF018F
:103320004A5F5F4F658170E084810E941F19089594
:1033300080818093EB0483E08093EC041092ED0491
:1033400083E090E00E94BD0108951F920F920FB696
:103350000F9211240F900FBE0F901F9018959C0193
:103360000897029718F024E030E017C0F901EB5BF2
:10337000FC4F8DE081832830310561F02930310523
:1033800019F027E030E009C0BD9A81E090E09BBDD4
:103390008ABD01C0BC9A21E030E0C9010895FC015A
:1033A000EB5BFC4F118281E090E008959C01FC01F1
:1033B000EB5BFC4F81818D3019F026E030E029C0B5
:1033C0002830310521F12930310519F027E030E0AE
:1033D00020C063307105A9F0643071053CF46130A0
:1033E000710559F06230710591F409C064307105BE
:1033F00051F06530710559F408C081E007C082E0E2
:1034000005C083E003C084E001C085E08EBD21E0FB
:1034100030E0C90108959C01FC01EB5BFC4F818108
:103420008D3019F026E030E00DC02830310541F034
:103430002930310519F027E030E004C07BBD6ABDBA
:1034400021E030E0C90108959C0183E58093EB04FD
:10345000F901EB5BFC4F81818D3019F086E090E043
:103460000DC02830310541F02930310519F087E0D1
:1034700090E004C07BBD6ABD81E090E08093EC04E5
:103480001092ED0483E090E00E94BD01089522E5D2
:103490002093EB040E94D6198093EC041092ED0463
:1034A00083E090E00E94BD01089521E52093EB04A4
:1034B000FC01EB5BFC4F118281E08093EC041092E5
:1034C000ED0483E090E00E94BD01089520E5209383
:1034D000EB040E94AF198093EC041092ED0483E09A
:1034E00090E00E94BD010895FC018081813579F052
:1034F000823518F48035F1F405C0823569F08335E2
:10350000C9F411C0828190E00E94661A08958281F8
:1035100090E00E94551A0895638170E0828190E0E6
:103520000E94471A0895638170E0828190E00E94B2
:10353000241A08958093EB0483E08093EC041092A6
:10354000ED0483E090E00E94BD010895DF93CF93E6
:10355000CDB7DEB7CF91DF910895089581E090E077
:10356000089508958A3310F4805301C087556A3353
:1035700010F4605301C067556F708295807F862B71
:1035800008950895DC0180E1A030B80710F082E0D2
:103590000895E199FECF9D0109C03FBB2EBB2F5F6F
:1035A0003F4FE09A8DB3E60FF71F8083822F8A1B6F
:1035B000E82FF0E0E417F50780F381E00895DC01DF
:1035C00080E1A030B80710F082E00895E199FECFC5
:1035D0009D010AC03FBB2EBB2F5F3F4FE60FF71F79
:1035E00080818DBBE29AE19A822F8A1BE82FF0E05E
:1035F000E417F50778F381E008950F931F938B018B
:1036000021E82093EB040E94DF1A8093EC041092CF
:10361000ED041F930F9389EF92E09F938F930E9485
:10362000A61A83E090E00E94BD010F900F900F90CA
:103630000F901F910F910895CF93DF93AC01EB0191
:1036400080E88093EB0480E14030580710F082E07E
:1036500015C0E199FECF9A0109C03FBB2EBB2F5F79
:103660003F4FE09A8DB3E351FB4F8083822F841B41
:10367000E82FF0E0EC17FD0780F381E08093EC0485
:10368000FE01E351FB4F10828DEE94E09F938F93E8
:1036900086E093E09F938F930E94A61ACE01039633
:1036A0000E94BD010F900F900F900F90DF91CF916E
:1036B0000895EF92FF920F931F93CF93DF93EC0146
:1036C0009B8180E02A817C01E20EF11C9D8180E0DB
:1036D0002C818C01020F111DFF92EF921F930F930B
:1036E00080E193E09F938F930E94A61A88812DB763
:1036F0003EB72A5F3F4F0FB6F8943EBF0FBE2DBFB7
:10370000803819F0813869F405C0B801C7010E94FA
:103710001C1B12C02696A801BE01C7010E94FD1AFB
:103720000BC08093EB0483E08093EC041092ED04D3
:1037300083E090E00E94BD01DF91CF911F910F9136
:10374000FF90EF900895CF93DF93BC0182309105F5
:1037500010F462E070E0A0917006B0917106ED0186
:10376000E0E0F0E040E050E021C0888199818617D8
:10377000970769F48A819B81309719F0938382833C
:1037800004C09093710680937006FE0133C06817E1
:10379000790738F44115510519F08417950708F495
:1037A000AC01FE018A819B819C01E9012097E9F629
:1037B00041155105A1F1CA01861B970B049708F426
:1037C000BA01E0E0F0E029C08D919C911197841737
:1037D0009507F1F46417750779F4ED018A819B81EF
:1037E000309719F09383828304C09093710680937D
:1037F0007006FD0132964CC0CA01861B970BFD0175
:10380000E80FF91F6193719302978D939C9340C0C9
:10381000FD01828193819C01D9011097A9F68091C5
:103820006E0690916F06892B41F480913703909139
:10383000380390936F0680936E0640913903509140
:103840003A034115510541F44DB75EB780913503F8
:1038500090913603481B590B20916E0630916F06EC
:10386000CA01821B930B8617970780F0AB014E5F4E
:103870005F4F8417950750F0420F531F50936F0608
:1038800040936E06F9016193719302C0E0E0F0E0AD
:10389000CF01DF91CF910895CF93DF93009709F483
:1038A0004EC0EC0122971B821A82A0917006B09143
:1038B0007106109701F140E050E0AC17BD0700F130
:1038C000BB83AA83FE0121913191E20FF31FAE1752
:1038D000BF0771F48D919C911197280F391F2E5FAE
:1038E0003F4F39832883FD01828193819B838A83A3
:1038F0004115510569F4D0937106C09370061FC03D
:10390000FD0182819381AD01009711F0DC01D5CFDB
:10391000FA01D383C28321913191E20FF31FCE17B5
:10392000DF0769F488819981280F391F2E5F3F4F87
:10393000FA01318320838A819B8193838283DF9183
:10394000CF91089597FB092E07260AD077FD04D062
:103950000CD006D000201AF4709561957F4F089521
:10396000F6F7909581959F4F0895AA1BBB1B51E1D7
:1039700007C0AA1FBB1FA617B70710F0A61BB70BDF
:10398000881F991F5A95A9F780959095BC01CD0184
:063990000895F894FFCF3A
:10399600456D62656464656450726F6A65637473CD
:1039A600004F63746F70757355534220496E74658A
:1039B600726661636520436F6E7665727465722008
:1039C600616E6420492F4F20457874656E73696F68
:1039D6006E003230303831313038006669727374B7
:1039E600207061636B6574206F662061206C6F6E5A
:1039F60067206D65737361676520286C656E6774F3
:103A0600683A202564290A006F63746F7075732005
:103A16006C6F6E672072756E6E696E67206D65736A
:103A2600736167650A006F63746F7075732E6C6FD0
:103A36006E675F696E646578203C206F63746F7093
:103A460075732E6C6F6E675F62797465730A006EAC
:103A56006F74206C617374207061636B65743A20B7
:103A660064696666203E2036340A006C61737420F1
:103A76007061636B65740A007061727365722C20E5
:103A8600636865636B3A2025582C20636F6D6D6102
:103A96006E643A2025580A0063616C6C696E672073
:103AA600696F5F7061727365720A0063616C6C693D
:103AB6006E67206164635F7061727365720A00638A
:103AC600616C6C696E67206932635F7061727365E1
:103AD600720A0063616C6C696E67207370695F704F
:103AE60061727365720A0063616C6C696E6720703F
:103AF600776D5F7061727365720A0063616E277419
:103B06002063616C6C2063616E5F706172736572B5
:103B1600202D206E6F2043414E2D737570706F728D
:103B2600740A0063616C6C696E6720656570726FFC
:103B36006D5F7061727365720A00756E6B6E6F777A
:103B46006E20636D640A00726563656976696E67E7
:103B560020636F6D6D616E643A20255820286C6570
:103B66006E6774683A202575290A00676574206EA9
:103B76006578740A0067657420616E6420657865EF
:103B8600637574650A000904007772697474656E5A
:103B96003A2025730A00726561643A2025730A008B
:103BA600656570726F6D5F7061727365723A206CD5
:103BB600656E6774683A2025752C20616464723AD4
:0C3BC6002025750A002000720600000097
:00000001FF
